:100000000C941E060C9488260C94B5260C94460677
:100010000C9446060C9446060C9446060C94460630
:100020000C9446060C9446060C94D5110C94460686
:100030000C9446060C9446060C9446060C94460610
:100040000C94E2260C9446060C94D02A0C94132BA4
:100050000C9446060C9446060C9446060C944606F0
:100060000C9446060C9446063117931772177517B1
:1000700078177B177E178117841793178D17C5186C
:10008000C718C718C518C718C718C718C718C7187A
:10009000C718C718C718C718C718C718C718C71868
:1000A0004B18C718C718C718C718C718BC17C718E0
:1000B000C718C718C718C718C718C718C718C71848
:1000C000C718C718C718C718C718C7185718571818
:1000D0005718571857185718571857185718C71838
:1000E000C718C718C718C718C718BC175618561806
:1000F00056185618C71864186A18701876187C189D
:10010000821888188E189818A218AC18B618FD17FF
:10011000BF17C718C718C718C7184B18C718C7186C
:10012000C718C718C718C718C718C71855185518BB
:1001300055185518C71864186A18701876187C185E
:10014000821888188E189818A218AC18B618FD17BF
:10015000BF17C718C718C718C7184B18FA18FA18C6
:10016000FA18FA18FA18FA18FA18FA18FA18FA18FF
:10017000FA18FA18FA18111A111A111A111A111A72
:10018000111A3F19491953195D19BB19C519D41909
:10019000E5196C1B811B8D1B961BA51BCA1BD31B52
:1001A0001C1CE51B131F191F1F1F261F341F561F62
:1001B000741F456E746572206D656E752E2E2E004F
:1001C000546F67676C6564206D6963726F50504D42
:1001D00000546F67676C656420696E76657274653C
:1001E000642050504D2100546F67676C6564205443
:1001F00058206D7574696E672100546F67676C6570
:10020000642074656C656D65747279210050726F3D
:10021000746F636F6C206572726F72207769746897
:100220002052580054696D656F7574207768656E4B
:1002300020636F6E6E656374696E6720746F205201
:100240005800507265737320616E79206B65792058
:10025000746F2063616E63656C00436F6E6E6563DF
:1002600074696E6720746F2052582C20706F776508
:100270007220757020746865205258202877697440
:10028000682062696E6420706C7567206966206EF4
:100290006F74207573696E6720616C776179732064
:1002A00062696E642900546F67676C656420276912
:1002B0006D6D656469617465206F75747075742700
:1002C00000546F67676C65642027736C61766520E6
:1002D0006D6F64652700546F67676C6564202761E4
:1002E0006C776179732062696E642700546F676769
:1002F0006C65642050504D206368616E6E656C20A3
:100300006C696D69740053657420525353492069B8
:100310006E6A656374696F6E206368616E6E656C8A
:100320002028303D3D64697361626C652900536526
:10033000742050504D206D696E696D756D20737914
:100340006E630053657420626561636F6E20696E31
:1003500074657276616C0053657420626561636FC9
:100360006E2064656C617900536574206265616319
:100370006F6E206672657175656E637920696E2097
:10038000487A3A20303D64697361626C652C205074
:10039000783D504D52206368616E6E656C20782CFC
:1003A0002046783D465253206368616E6E656C202E
:1003B00078005365742050574D2073746F7020641B
:1003C000656C61792028302064697361626C6564B2
:1003D0002C20312D323535203D3D20302E317320FB
:1003E0002D2035306D696E29005365742050504DB5
:1003F0002073746F702064656C61792028302064EC
:10040000697361626C65642C20312D323535203D75
:100410003D20302E3173202D2035306D696E29003E
:10042000536574206661696C736166652064656CF0
:1004300061792028302064697361626C65642C20C6
:10044000312D323535203D3D20302E3173202D2089
:1004500035306D696E29002A2A2A2A2A2A2A2A2A50
:100460002A2A2A2A2A2A2A2A2A2A2A2A2A2A2A2AEC
:100470002A2A2A2A0052582041636B6564202D20C5
:1004800072657665727420737563636573736675E0
:100490006C21002A2A2A2A2A2A2A2A2A2A2A2A2AAD
:1004A0002A2A2A2A2A2A2A2A2A2A2A2A2A2A2A2AAC
:1004B000002A2A2A2A2A2A2A2A2A2A2A2A2A2A2AC6
:1004C0002A2A2A2A2A2A2A2A2A2A2A2A2A2A00528E
:1004D000582041636B6564202D20757064617465DC
:1004E000207375636365737366756C21002A2A2A0D
:1004F0002A2A2A2A2A2A2A2A2A2A2A2A2A2A2A2A5C
:100500002A2A2A2A2A2A2A2A2A2A0056616C696457
:100510002063686F69636573206172653A205B319F
:100520005D2D5B31365D20286368616E6E656C20E1
:10053000312D31362900536574206F7574707574D0
:1005400020666F7220706F727420005B585D2061AE
:10055000626F7274206368616E67657320616E6498
:10056000206578697420525820636F6E6669670051
:100570005B535D20736176652073657474696E6783
:100580007320746F205258005B525D20726576654F
:1005900072742052582073657474696E6773207486
:1005A0006F2064656661756C747300557365206EA9
:1005B000756D62657273205B312D445D20746F2010
:1005C0006564697420706F727473205B452D515D92
:1005D00020666F722073657474696E677300202DD6
:1005E00020726563656976657220636F6E66696700
:1005F000757261746F722C20727820737720000AF4
:100600000A6F70656E4C52536E67200053657420FC
:1006100073657269616C2062617564726174653AB8
:10062000200056616C69642063686F696365733A82
:100630002031202D20342B34202F2032202D203823
:10064000202F2033202D20382B34202F2034202D14
:10065000203132202F2035202D2031322B34202FF5
:100660002036202D20313600536574204368616E9A
:100670006E656C20636F6E6669673A20005365741F
:100680002044617461726174652028302D32293AEA
:10069000200053657420486F70206368616E6E653A
:1006A0006C7320286D61782032342C207365706162
:1006B000726174656420627920636F6D6D61732966
:1006C0002076616C69642076616C75657320312DCC
:1006D0003235353A2000536574206368616E6E656B
:1006E0006C2073706163696E6720287831306B48C5
:1006F0007A293A200053657420524620706F77653E
:10070000722028302D37293A200053657420524634
:10071000206D6167696320286865782920652E67E8
:100720002E20307844454144463030443A2000532E
:1007300065742062617365206672657175656E63AC
:10074000792028696E20487A293A20005B5A5D207A
:10075000656E746572207265636569766572206383
:100760006F6E66696775726174696F6E2075746902
:100770006C79005B465D20646973706C61792061FF
:10078000637475616C206672657175656E63696509
:10079000732075736564005B525D2063616C6375E3
:1007A0006C6174652072616E646F6D206B65792079
:1007B000616E6420686F70206C697374005B495DC2
:1007C000207265696E697469616C697A6520736508
:1007D0007474696E677320746F20736B65746368DB
:1007E0002064656661756C7473005B585D2072658A
:1007F00076657274206368616E67657320616E64EC
:100800002065786974206D656E75005B535D20739B
:100810006176652073657474696E677320746F20E8
:10082000454550524F4D20616E64206578697420B3
:100830006D656E7500557365206E756D62657273BA
:10084000205B302D395D20746F20656469742070E1
:100850006172616D657465727300202D2053797328
:1008600074656D20636F6E66696775726174696F18
:100870006E000A0A6F70656E4C52536E672000510D
:1008800029204F7574707574206265666F726520DB
:100890006C696E6B20283D465329203A2000502970
:1008A00020536C617665206D6F64652028657870D3
:1008B0006572696D656E74616C293A20004F29205C
:1008C00054696D65642042494E44206174207374FC
:1008D000617274757020203A20004E292050504DCE
:1008E000206F7574707574206C696D69746564200F
:1008F000202020203A200044495341424C454400E6
:100900004D292050504D205253534920746F20637D
:1009100068616E6E656C202020203A20004C2920F2
:1009200050504D206D696E696D756D2073796E63E1
:10093000202875732920203A200044495341424C15
:100940004544004B29204661696C736166652062ED
:100950006561636F6E20696E74762E2028312D32AA
:10096000353573293A20004A29204661696C736144
:10097000666520626561636F6E2064656C617920D5
:1009800028302D323535203D3E20313073202D204A
:100990003135306D696E293A200049292046616958
:1009A0006C7361666520626561636F6E206672714B
:1009B0002E203A200048292050574D2073746F7024
:1009C0002064656C6179202020202020203A2000BE
:1009D00047292050504D2073746F702064656C61FE
:1009E00079202020202020203A200046292046611E
:1009F000696C736166652064656C617920202020D4
:100A00002020203A200050574D206368616E6E65AB
:100A10006C200066756E6374696F6E3A2000292041
:100A2000706F72742000506F776572546F776572C3
:100A300000445446205548462033322D62697420C4
:100A400031306368004F70656E4C52536E67525878
:100A5000206D696E6920342F36636800466C7974A6
:100A6000726F6E2F4F72616E6765525820554846FF
:100A70002038636800525820747970653A20004429
:100A8000697361626C656400487A00203D3D200016
:100A900043616C63756C61746564207061636B6540
:100AA0007420696E74657276616C3A200042292068
:100AB0004D6963726F202868616C66292050504D23
:100AC000202020203A00412920496E766572746505
:100AD000642050504D20696E20202020203A0030A4
:100AE00029204D7574652062757A7A657220286DAB
:100AF0006F73746C79293A003929205365726961E2
:100B00006C2062617564726174653A00736D617224
:100B100074506F7274004672536B79005472616E38
:100B200073706172656E740044697361626C6564B0
:100B30000038292054656C656D657472793A2020FF
:100B40002020202020003729204368616E6E656CCC
:100B500020636F6E6669673A202000362920446161
:100B60007461726174652028302D32293A2020206A
:100B700000352920486F70206368616E6E656C7364
:100B80003A2020202020003429204368616E6E65C1
:100B90006C2073706163696E673A202000332920EE
:100BA000524620706F7765722028302D37293A2001
:100BB0002020003229205246206D616769633A2067
:100BC0002020202020202020003129204261736530
:100BD000206672657175656E63793A202020000089
:100BE00000000700020100000304060000000000EE
:100BF00000000001020408102040800102040810D7
:100C00002001020408102004040404040404040263
:100C10000202020202030303030303000000002395
:100C2000002600290000000000250028002B0000FD
:100C3000000000240027002A0000012C11241FBE00
:100C4000CFEFD8E0DEBFCDBF13E0A0E0B1E0E0E140
:100C5000FEE502C005900D92AA39B107D9F716E05A
:100C6000AAE9B3E001C01D92AF35B107E1F71CE07E
:100C7000CCE3DCE004C02297FE010E940A2DCA33B7
:100C8000D107C9F70E943D2C0C94062F0C9400004C
:100C90008091A505813019F482E08093A5058091AB
:100CA000A505833019F484E08093A5050895A895DF
:100CB0000895DC01ED91FC910190F081E02D099502
:100CC000089561E08FE00E94E52760E08FE00E94D8
:100CD0001E280895892B11F061E001C060E08FE0CB
:100CE0000E941E28089560E08CE00E94E52761E0E4
:100CF0008BE00E94E52761E08DE00E94E52760E03F
:100D000082E00E94E52761E084E00E94E5270895E3
:100D100042E050E068E476E080E00E9468260895B2
:100D2000E3E0F0E089E080935700E491E67081E031
:100D3000E63009F080E00895CF93DF93C82F0E943A
:100D40009006882381F0DFB781E08093A405F894B2
:100D50000E94570688E180936000C0936000C11133
:100D60000E945706DFBFDF91CF910895209144057F
:100D700030914505382748E0C901880F991F37FF92
:100D800006C09C0151E2252750E1352701C09C0196
:100D9000415091F730934505209344050895D82F8D
:100DA000C0E0CD1790F45E9A409A64E670E080E06F
:100DB00090E00E945B275E98409864E670E080E0D7
:100DC00090E00E945B27CF5FECCF6CE271E080E0A7
:100DD00090E00E945B27E4CF0F931F93CF93DF93A4
:100DE000EC01062F15E0115051F0CE010E94ED2EBE
:100DF000081741F0602FCE010E94F52EF4CF82E05B
:100E00000E94CF06DF91CF911F910F910895A0E02E
:100E1000B0E0EDE0F7E00C94D32C482E562EC0E065
:100E2000D0E0612C712CE12CF12C00E010E041109D
:100E30000CC06090A30586E4689E30011124A9E1EE
:100E4000EA2EF12C0AE815E01EC091E049120FC00D
:100E50006090A305E6E46E9E30011124FBE16F0E65
:100E6000711CF9E2EF2EF12C06E415E00CC082E0D3
:100E7000481209C078E1672E77247394EE24E39436
:100E8000F12C03EA15E043018C0E9D1E10924505DE
:100E9000109244053401A62CA818B12CC301019668
:100EA0006C01AE14BF04A8F4A00EB11E511006C010
:100EB000C3010E94ED2EF501808305C0F50160811C
:100EC000C3010E94EC06F50180810E94B60636013E
:100ED000E2CFC301511018C0C3010E94ED2EB82EFD
:100EE000C6010E94ED2E2B2D30E0322F2227282B19
:100EF00080914405909145058217930779F4C0E0ED
:100F0000D0E05524539493CF3601609145050E945B
:100F1000EC0660914405C6010E94EC06C05EDE4FFF
:100F2000C13E92E0D90708F482CF852DCDB7DEB758
:100F3000E0E10C94EF2C87E38093460580E092EC8F
:100F4000A1E0B0E08093470590934805A093490540
:100F5000B0934A0587E08093530580EC92E9ADEEAB
:100F6000B9E180934B0590934C05A0934D05B09348
:100F70004E0585E0809354058DEE9EEFADEABEED03
:100F800080934F0590935005A0935105B09352055F
:100F9000E5E5F5E080E090E0863028F4DC01AC592E
:100FA000BC4F2C9101C020E021930196883191051E
:100FB00099F782E080936D058AE080936E0508952D
:100FC00061E082E00E940707089560E082E00E94ED
:100FD00007078091A305843020F01092A3050E949A
:100FE000E0070895A1E0B0E0E8EFF7E00C94E12C11
:100FF00089830E94E5079091A3058981981731F0B4
:10100000843020F48093A3050E94E0072196E2E05B
:101010000C94FD2C80EC91EDA8E9BBE180938B054D
:1010200090938C05A0938D05B0938E0580E090E0A1
:10103000A0E0B0E580938F0590939005A093910573
:10104000B0939205E3E9F5E080E081938F5F803112
:10105000E1F70895A0E0B0E0E0E3F8E00C94D72CCD
:101060000E9438276115710581059105C9F30E9419
:10107000762D10924F051092500510925105109246
:101080005205C4E0C12CD12C7601CA9480904F0542
:1010900090905005A0905105B0905205BA2CA92C03
:1010A000982C88240E94712DA70196010E94B22CD1
:1010B000680D791D8A1D9B1D60934F057093500527
:1010C0008093510590935205C15001F705E515E055
:1010D000E801C12CD12CB2E38B2E912CA12CB12C88
:1010E00080E1E82E87E2F82E8881882309F446C043
:1010F000D39419F40E949B0741C00E94712DA50151
:1011000094010E94B22C21E0260FE5E5F5E08E2F38
:10111000801B8C1520F481918213F9CFE9CF409187
:101120005405249FA00111244E9DC0014F9D900D98
:101130005E9D900D1124AA2797FDA095BA2F40918E
:101140004B0550914C0560914D0570914E05840FF3
:10115000951FA61FB71F40918B0550918C0560917C
:101160008D0570918E05481759076A077B0708F4AB
:10117000BFCF2993C39488E1C812B6CFCDB7DEB7ED
:10118000ECE00C94F32C61E080E00E94070761E042
:1011900081E00E940707089560E080E00E94070751
:1011A000882331F060E081E00E940707811108C0C8
:1011B0000E940A080E949B070E942A080E94C308F6
:1011C00008958436910520F4BC0180E090E017C0BA
:1011D0009C018E3B910528F42A553109AAE0B0E024
:1011E0000CC0823D910528F4245B3109A4E6B0E0EF
:1011F00004C02D5C3109A8E5B2E00E944A2CA4E6A7
:10120000B0E09B01AC010E94592C089590E08C59EC
:101210009F4F0E94E10808958F929F92AF92BF92D4
:10122000CF92DF92EF92FF92CF93FC01C0A5EC2FFB
:10123000E770F0E0E45BFC4FA081B0E0C7FF03C0C3
:1012400024E130E002C02FE030E0FC0197A183E10F
:10125000989FF0011124E25CFE4F80809180A28073
:10126000B380A20FB31F20E43FE14DE750E00E949E
:10127000642CA50194010E94902C8C2F887149F454
:1012800069017A01E0EDCE0EE7E0DE1EE11CF11C03
:101290001BC0C7FF05C060E47AE88CE29EE004C092
:1012A00060E07EEE8AEB9BE069017A01F8EBCF0EFD
:1012B000FBE0DF1EE11CF11CA50194010E94902CB3
:1012C000C20ED31EE41EF51EC701B60169517C4F44
:1012D0008F4F9F4F28EE33E040E050E00E94902C6B
:1012E000A8EEB3E00E94592CCF91FF90EF90DF90D1
:1012F000CF90BF90AF909F908F9008958F3F9105B2
:1013000051F048F0811522E0920738F081159340A2
:1013100030F482E0089580E0089581E0089583E04C
:101320000895A0E0B0E0E7E9F9E00C94DC2CEB01D3
:101330008A01B82FB695A0E028813981F801208371
:101340002A813B8121832C813D8122832E813F8113
:101350002383688179814A815B812C813D81EE8183
:10136000FF819F2F9295990F990F907C272F2370C3
:10137000922B252F2370220F220F922B232F2370C5
:101380002295207F922BF80194830B5F1F4F2896A4
:10139000AF5FBA1788F680FF24C0888199810E94C8
:1013A0007E09D82E8A819B810E947E09E82E8C813D
:1013B0009D810E947E09F82E8E819F810E947E0968
:1013C000F0E4DF9EA001112490E1E99E9001112438
:1013D000242B282BE4E0FE9EB0011124262BF801DB
:1013E0002083CDB7DEB7E7E00C94F82C803223E001
:1013F000920708F1883E23E0920740F48F51934012
:10140000E4E096958795EA95E1F70895803D27E019
:10141000920718F48C5D93400895883928E092076C
:1014200068F4885C974074E0969587957A95E1F723
:101430008D509C4F089580E090E008958FEF93E0E9
:1014400008958C30910540F4A4E0880F991FAA9567
:10145000E1F7885D9C4F0895843F23E0920718F4DC
:1014600084529C4F0895811524E0920740F48657DA
:10147000934FF4E0880F991FFA95E1F7089580E9FA
:1014800098E008959C013695279525753575821B42
:10149000930B9C0123733373969587959695879547
:1014A00083739373820F931F9C0154E036952795A5
:1014B0005A95E1F7280F391F2F703F7041E051E036
:1014C000249FC001259F900D349F900D1124892FDA
:1014D00008952D98882319F000002B9A02C000006F
:1014E0002B9800002D9A000008952D9A000083B1DA
:1014F0002D980000829581700895CF93DF93D82FA7
:101500005C9A2D985C98C8E08D2F80780E94690ABB
:10151000DD0FC150C9F72D98DF91CF9108958F77D6
:101520000E947D0A0895CF93DF93D82FC8E08D2FB6
:1015300080780E94690ADD0FC150C9F72D98DF91AC
:10154000CF910895CF93DF932D98C8E080E0D82FF6
:10155000DD0F0E94750A8D0FC150C9F7DF91CF9141
:1015600008950E948F0A0E94A20A5C9A0895A1E041
:10157000B0E0EDEBFAE00C94E12C806869830E9406
:101580007D0A6981862F0E94930A5C9A2196E2E087
:101590000C94FD2CCF93C0914F05C827E82FF0E0A5
:1015A000EA5BFA4F678589E70E94B70A6C2F8DE3E3
:1015B0000E94B70A6C2F82E40E94B70ACF91089567
:1015C00086E20E94B10A0895CF93DF93EC016C810B
:1015D0008CE10E94B70A6D818DE10E94B70A6E818D
:1015E0008EE10E94B70A6F8180E20E94B70A688587
:1015F00081E20E94B70A698582E20E94B70A6A8581
:1016000083E20E94B70A6B8584E20E94B70A6C8568
:1016100085E20E94B70A6D858AE20E94B70A6E854C
:101620008EE60E94B70A6F858FE60E94B70A688926
:1016300080E70E94B70A698981E70E94B70A6A8930
:1016400082E70E94B70ADF91CF910895CF92DF928F
:10165000EF92FF92CF93DF936B017C01C11488E37B
:10166000D8068CE9E8068CE1F80628F5C701B60132
:1016700020E836E948E950E00E94902CE90168979B
:1016800060E879E687E69FEF0E946C2C6C0D7D1D6B
:101690008E1D9F1DF2E0660F771F881F991FFA9518
:1016A000D1F721E732E040E050E00E94902CF22E8A
:1016B000E32E80E421C0C701B60120E03DE241E312
:1016C00051E00E94902CE901689760E073ED8EEC88
:1016D0009EEF0E946C2C6C0D7D1D8E1D9F1D660F54
:1016E000771F881F991F21E732E040E050E00E94F9
:1016F000902CF22EE32E80E66C2F6F71680F85E739
:101700000E94B70A6E2D86E70E94B70A6F2D87E701
:101710000E94B70ADF91CF91FF90EF90DF90CF90BA
:101720000895682F8DE60E94B70A08958F929F92C0
:10173000AF92BF92CF92DF92EF92FF92CF93DF935F
:10174000D82F83E00E94B10A8093430584E00E9471
:10175000B10A8093420560E086E00E94B70A61E02A
:1017600087E00E94B70A6FE789E00E94B70A65E048
:101770008AE00E94B70A62E18BE00E94B70A65E145
:101780008CE00E94B70A6DEF8DE00E94B70A60E01E
:101790008EE00E94B70ADD2319F08BE291E008C0C9
:1017A00020916D0533E1239FC0011124825C9E4F7F
:1017B0000E94E40A6CE880E30E94B70A6FE082E3CB
:1017C0000E94B70A62E483E30E94B70A80916E0523
:1017D00087FF02C064E101C06AE084E30E94B70AA7
:1017E0006AE285E30E94B70A6DE286E30E94B70AC7
:1017F00064ED87E30E94B70A60E088E30E94B70ABD
:1018000060E089E30E94B70AD11109C0C0904F057A
:10181000D0905005E0905105F090520507C0C5E802
:10182000CC2EC1ECDC2EED2CCEEDFC2ECAE38F2CA1
:101830009924AA24BB24682D8C2F0E94B70A682DF6
:1018400085E08C0F0E94B70AFE2CED2CDC2CCC24FA
:10185000CF5FCE3361F76FEF83E40E94B70A6FEF7B
:1018600084E40E94B70A6FEF85E40E94B70A6FEF25
:1018700086E40E94B70ADD2311F066E002C06091A1
:1018800053058DE60E94B70A60E089E70E94B70A17
:10189000609154058AE70E94B70A60E083E70E94DE
:1018A000B70A60E084E70E94B70AD11109C06091CD
:1018B0004B0570914C0580914D0590914E0504C0EB
:1018C00060EC72E98DEE99E10E94260BDF91CF91D9
:1018D000FF90EF90DF90CF90BF90AF909F908F9050
:1018E000089561E087E00E94B70A64E28EE70E94F3
:1018F000B70A63E088E00E94B70A60E088E00E94CF
:10190000B70A65E087E00E94B70A62E085E00E94BE
:10191000B70A83E00E94B10A8093430584E00E94E5
:10192000B10A80934205089583E00E94B10A809332
:10193000430584E00E94B10A8093420561E087E09C
:101940000E94B70A6AE070E080E090E00E945B27A6
:101950000E94710C00000895CF92DF92FF920F93C6
:101960001F93CF93DF931F92CDB7DEB7082F162FAB
:101970008EE399830E94B70AF02EC02E9981D92E4A
:101980008C2D8F19811738F4F60161916F018FE763
:101990000E94B70AF5CF64E085E00E94B70A83E0B1
:1019A0000E94B10A8093430584E00E94B10A8093AB
:1019B00042050E94382760933E0570933F0580934F
:1019C00040059093410569E087E00E94B70A81E0F5
:1019D0008093A5050F90DF91CF911F910F91FF90FC
:1019E000DF90CF9008950F931F930E94AC0C8091CD
:1019F000A505813099F40E94382700913E05109189
:101A00003F052091400530914105601B710B820B11
:101A1000930B603A76488140910548F38091A50583
:101A2000813031F46EE971E083EB95E00E94242966
:101A30001F910F9108950F931F938091A5058230F8
:101A400021F41092A50581E020C08091A505813088
:101A5000D9F40E94382700913E0510913F0520914E
:101A6000400530914105601B710B820B930B613A6D
:101A700076488140910540F061E087E00E94B70A16
:101A80001092A50582E001C080E01F910F9108959A
:101A9000CF93DF93EC014AE050E06D2F70E083EBD1
:101AA00095E00E94F2296EE283EB95E00E94F62811
:101AB000BE0184E0769567958A95E1F76F70772788
:101AC0004AE050E083EB95E00E94F2296EE283EB5E
:101AD00095E00E94F628BE016F7077274AE050E03B
:101AE00083EB95E00E94F229DF91CF91089588233E
:101AF00019F06AEA71E002C06EEA71E083EB95E0EA
:101B00000E9424290895FF920F931F93CF93DF9390
:101B100069EC7BE083EB95E00E94D02840914B0577
:101B200050914C0560914D0570914E052AE030E0D2
:101B300083EB95E00E94F92963EB7BE083EB95E072
:101B40000E94D02840914F05509150056091510559
:101B50007091520520E130E083EB95E00E94F92975
:101B60006DE97BE083EB95E00E94D0284AE050E0ED
:101B70006091530583EB95E00E94212A67E87BE0A2
:101B800083EB95E00E94D0284AE050E06091540534
:101B900083EB95E00E94212A61E77BE083EB95E0EF
:101BA0000E94D028C5E5D5E0F12C8E0188818823DC
:101BB000A9F0FF2031F061EB71E083EB95E00E942A
:101BC000F32821964AE050E0F801608183EB95E02C
:101BD0000E94EA29F394F8E1FF12E7CF83EB95E046
:101BE0000E94FE286BE57BE083EB95E00E94D02805
:101BF0004AE050E060916D0583EB95E00E94212A58
:101C000066E47BE083EB95E00E94D028E0916E05CE
:101C1000E770F0E0EE0FFF1FEC5AFC4F608171811E
:101C200083EB95E00E94242961E37BE083EB95E060
:101C30000E94D02880916E058871883069F028F460
:101C4000811113C068E27BE00CC0803141F0883123
:101C500061F46CE07BE005C06CE17BE002C066E112
:101C60007BE083EB95E00E94122968EF7AE083EB3A
:101C700095E00E94D0284091470550914805609119
:101C8000490570914A052AE030E083EB95E00E9417
:101C9000F9296FED7AE083EB95E00E94D0288091DE
:101CA0008F0580710E94770D66EC7AE083EB95E0FA
:101CB0000E94D02880918F0580740E94770D6DEA74
:101CC0007AE083EB95E00E94D02880918F058072A6
:101CD0000E94770D60E97AE083EB95E00E94D028BE
:101CE00086E495E00E940C09AB01BC012AE030E0DB
:101CF00083EB95E00E94DB296BE87AE083EB95E0CB
:101D00000E94D02886E495E00E940C099B01AC015A
:101D100060E472E48FE090E00E94902CBA01A90187
:101D20002AE030E083EB95E00E94DB2968E87AE066
:101D300083EB95E00E941229CDB7DEB7E5E00C9465
:101D4000FA2C8F929F92AF92BF92CF92DF92EF9236
:101D5000FF92811107C06FE77AE083EB95E00E9464
:101D600012292FC090E00E94E10824E630E040E014
:101D700050E00E94902CCA01B9012AE030E040E016
:101D800050E00E94902C49015A016B017C012AE02D
:101D900030E0B501A40183EB95E00E94DB296EE2FF
:101DA00083EB95E00E94F6282AE030E0B701A60117
:101DB00083EB95E00E94DB2963E783EB95E00E94CB
:101DC0003629FF90EF90DF90CF90BF90AF909F901B
:101DD0008F9008951F93CF93DF9365E77AE083EBAD
:101DE00095E00E94D02880916F05813041F46CE528
:101DF0007AE083EB95E00E94122910E050C0823017
:101E000019F465E47AE0F5CF843019F461E37AE0FF
:101E1000F0CF853091F766E27AE0EBCFC12FD0E0CA
:101E2000C930D1050CF441C068E3610F83EB95E044
:101E30000E94F6286EE17AE083EB95E00E94D028BC
:101E4000BE016F5F7F4F4AE050E083EB95E00E9458
:101E5000BA2963E17AE083EB95E00E94D028C1596A
:101E6000DA4FE981E03218F566E07AE083EB95E03D
:101E70000E94D0288981803130F06FE373E083EBDA
:101E800095E00E94F32869816F7070E06F5F7F4F6B
:101E90004AE050E083EB95E00E94C3291F5F8091E8
:101EA0001A05181708F4BACF0FC061E3BECFEF7060
:101EB000F0E0EE0FFF1FE659FC4F6081718183EB6C
:101EC00095E00E942429EACF6BEE79E083EB95E060
:101ED0000E94D028809187050E94A10E60ED79E0D4
:101EE00083EB95E00E94D028809188050E94A10E86
:101EF00065EB79E083EB95E00E94D028809189051D
:101F00000E94A10E6AE979E083EB95E00E94D02857
:101F100040917F0550918005609181057091820507
:101F2000411551056105710539F12AE030E083EB77
:101F300095E00E94F92967E679E083EB95E00E943D
:101F4000D028809183050E940609AB01BC012AE0DC
:101F500030E083EB95E00E94F92963E479E083EBBC
:101F600095E00E94D0284AE050E06091840583EB20
:101F700095E00E94212A06C06AE379E083EB95E0B0
:101F80000E9412296DE179E083EB95E00E94D02850
:101F900060918505709186054AE050E083EB95E0FD
:101FA0000E940B2A60E079E083EB95E00E94D02844
:101FB00060917E05603450F470E06F5F7F4F4AE0BF
:101FC00050E083EB95E00E94C32906C067EF78E0FC
:101FD00083EB95E00E9412296AED78E083EB95E0AF
:101FE0000E94D02880917D0580FF03C063EB71E0E3
:101FF00002C067EB71E083EB95E00E9424296DEB52
:1020000078E083EB95E00E94D02880917D05827076
:102010000E94770D6EE978E083EB95E00E94D0286E
:1020200080917D0584700E94770D6FE778E083EBE7
:1020300095E00E94D02880917D0588700E94770DE0
:10204000DF91CF911F9108950F931F93CF93DF934B
:10205000209117052F3FA9F56FEF75E083EB95E011
:102060000E94D02884E793E00E94480D6EED75E051
:1020700083EB95E00E94D028809118059091190576
:102080000E94480D6BEA75E083EB95E00E941229EF
:1020900068E875E083EB95E00E94122960E775E03F
:1020A00083EB95E00E9412296BE475E083EB95E0E9
:1020B0000E94122983EB95E00E94FE280E94EA0EFE
:1020C00068C012160CF065C0332727FD309580914B
:1020D0001A0590E0821793070CF45BC066E375E085
:1020E00083EB95E00E94D02860911705772767FD64
:1020F00070954AE050E083EB95E00E94C3296BE0C5
:1021000075E083EB95E00E94D02810E008E2809112
:102110001B051817D0F5C12FD0E0CC0FDD1FC45E12
:10212000DA4F288130E080911705992787FD909537
:1021300001972817390739F56BEB71E083EB95E0D0
:102140000E94F3284AE050E0602F83EB95E00E9464
:10215000EA296FEB71E083EB95E00E94F328E981B7
:10216000EF70F0E0EE0FFF1FE659FC4F60817181C8
:1021700083EB95E00E94F32863EC71E083EB95E03C
:102180000E94F3280F5F1F5FC2CF83EB95E00E9490
:10219000FE28DF91CF911F910F910895FF920F9329
:1021A0001F93CF93DF93C5E5D5E0F12C8E01888195
:1021B0008823D1F165EC71E083EB95E00E94F32870
:1021C0004AE050E06F2D83EB95E00E94EA2962ED32
:1021D00071E083EB95E00E94F3282196F8012081BD
:1021E00030E0A0E1B7E20E944A2C9B01AC01A09133
:1021F0005405B0E00E94592CAB01BC0180914B0505
:1022000090914C05A0914D05B0914E05480F591F76
:102210006A1F7B1F2AE030E083EB95E00E94F929DA
:10222000F394F8E1FF12C2CFCDB7DEB7E5E00C942E
:10223000FA2C1092B10485E6E2EBF4E0DF011D9286
:102240008A95E9F70895CF93C82F8F3719F0883012
:1022500009F045C0E091B104EE23D9F1E150E093DB
:10226000B104F0E0EE54FB4F10826DE070E083EBC0
:1022700095E00E945906C0E08091B104C81760F44F
:10228000EC2FF0E0EE54FB4F608170E083EB95E0C3
:102290000E945906CF5FF0CF60E270E083EB95E0DB
:1022A0000E9459066DE070E083EB95E00E945906AC
:1022B000C0E08091B104C81778F5EC2FF0E0EE543F
:1022C000FB4F608170E083EB95E00E945906CF5F81
:1022D000F0CF67E083EB95E00E94F6281DC08B31BC
:1022E00019F40E9419111AC08D30C1F08A30B1F072
:1022F0008091B104843668F76C2F70E083EB95E031
:102300000E945906E091B10481E08E0F8093B104E0
:10231000F0E0EE54FB4FC08380E001C081E0CF913C
:102320000895CF93C82F0E94382760939A04709322
:102330009B0480939C0490939D04C093AF04CC2392
:1023400029F040E051EE60E070E004C040E855E262
:1023500060E070E083EB95E00E94802BCF910895C0
:1023600090919E04492F4F7050E0BA016F5F7F4FEC
:10237000292F30E0E4E035952795EA95E1F76217DB
:10238000730759F0FA01E156FB4F808381E0890F12
:102390008F70907F892B80939E0408956EE770E084
:1023A00083EB95E00E94590608951F920F920FB695
:1023B0000F9211241F932F933F934F935F936F932B
:1023C0007F938F939F93AF93BF93CF93DF93EF93BD
:1023D000FF93C0918600D09187008091590490911D
:1023E0005A0420917B04211155C09E01281B390BF2
:1023F00080918F0590919005A0919105B0919205E3
:1024000085FD02C036952795253C49E03407B8F193
:1024100040910A0150E060E070E01CE1B695A7959C
:10242000979587951A95D1F70097A105B10521F4E5
:1024300081E090E0A0E0B0E084179507A607B70719
:10244000D8F480910A018F3FB9F040E080910A01F1
:10245000481780F4842F90E0880F991FFC01E55AFB
:10246000FB4F20813181FC01E55FFE4F31832083EA
:102470004F5FECCF10927C0410920A010BC02D3BF1
:1024800082E0380720F080910A018031D8F08FEF88
:1024900080930A01D0935A04C0935904FF91EF919D
:1024A000DF91CF91BF91AF919F918F917F916F916C
:1024B0005F914F913F912F911F910F900FBE0F9001
:1024C0001F90189510910A0181E0810F80930A01F5
:1024D000C9010E94F609E12FF0E0EE0FFF1FE55A57
:1024E000FB4F91838083D6CF83E0809380008AE97D
:1024F0008093810080918F0586FD05C080918100C9
:102500008064809381008FEF9FEF90938900809388
:10251000880080916F00806280936F0008956F3013
:1025200018F086958058089589E0689F802D1124C1
:102530000895A0E0B0E0EFE9F2E10C94DB2CC82FA5
:102540000E94382700910A0410910B0420910C047A
:1025500030910D046B017C01C01AD10AE20AF30A22
:102560009701860149E8C41643E1D406E104F10469
:1025700010F010920E0460930A0470930B04809381
:102580000C0490930D0420917B048FEF820F823016
:10259000D8F5E0910E04EE2309F44EC1E13011F4B8
:1025A00082E0B8C1E03108F034C181E08E0F809341
:1025B0000E04F0E0E55AFB4FC083803109F0ACC156
:1025C000EDE5F4E0213029F4A181A695A69580815E
:1025D00008C080819181A92FA695A695A69596956C
:1025E0008795A03148F4B0E090E0AA0FBB1FA55F2B
:1025F000BE4F11969C938E9310927C04329684E089
:10260000EB36F807F9F688C1233009F005C1E091EF
:102610000E04E11104C0CF3009F07EC10DC1E831D4
:1026200048F481E08E0F80930E04F0E0E65AFB4FF1
:10263000C08372C1E83109F0ECC0C111EAC040E0CA
:1026400050E0ABE0CA01B3E0880F991FBA95E1F7FB
:10265000A49F9001A59F300D1124F901E55AFB4F6D
:102660006081E1817E2F777075956795FC01EE0F93
:10267000FF1FE55FFE4F71836083F901E45AFB4F52
:10268000B081B695B695B695E181FE2FF295FF0F14
:10269000F07E6F2F6B2BE695E695E6957E2F777093
:1026A00075956795FC01EE0FFF1FE35FFE4F718389
:1026B0006083F901E35AFB4FB081B295B695B695A8
:1026C000B370C181DC2FDD0FDD0F6D2F6B2BC29539
:1026D000C695C695C370E281E170EE0FEE0F7E2FB6
:1026E0007C2B75956795FC01EE0FFF1FE15FFE4F98
:1026F00071836083F901E15AFB4FB081B695E181A6
:10270000FE2FF795FF27F7956F2F6B2BE6957E2F02
:10271000777075956795FC01EE0FFF1FEF5EFE4F1A
:1027200071836083F901E05AFB4FB081B295BF70AD
:10273000E181FE2FF295F07F6F2F6B2BE295EF700A
:102740007E2F777075956795FC01EE0FFF1FED5E8C
:10275000FE4F71836083F901EF59FB4FB081BB1FBE
:10276000BB27BB1FC181DC2FDD0F6D2F6B2BCC1F57
:10277000CC27CC1FE281E370EE0F7E2F7C2B75956A
:102780006795FC01EE0FFF1FEB5EFE4F71836083C8
:10279000F901ED59FB4FB081B695B695E181FE2F59
:1027A000F295FF0FFF0FF07C6F2F6B2BE695E695F0
:1027B0007E2F777075956795FC01EE0FFF1FE95E20
:1027C000FE4F71836083F901EC59FB4F2081229504
:1027D000269527703181E32FEE0FEE0FEE0F6E2F4F
:1027E000622B732F72957695777075956795FC01BE
:1027F000EE0FFF1FE75EFE4F718360834F5F5F4FF9
:102800004230510509F01ECF8091710483FF109270
:102810007C0410920E0480C0243009F07DC06091C9
:102820000E0461110BC0C83AB1F410924505109224
:10283000440588EA0E94B60681E06CC0613019F454
:10284000C093090404C0623031F4C09308048C2F93
:102850000E94B6065AC0E09108042E2F30E0220FE5
:10286000331F462F50E0C9010296841795073CF0AC
:10287000633268F7FA01E85AFB4FC083E8CF2D5F57
:102880003F4F8C2F90E060914405709145054217B1
:10289000530749F4982F8827862797279093450553
:1028A0008093440532C06817790769F5809109045F
:1028B000813049F5E13118F080E180930804F0900F
:1028C0000804CCE5D4E000E010E00F15D0F4FE01E0
:1028D0003197808190E0982F88272881822B63E0B0
:1028E000969587956A95E1F70E94F609F801EE0F33
:1028F000FF1FE55FFE4F918380830F5F1F4F22967E
:10290000E4CF10927C0410920E0480910E04882370
:1029100019F08F5F80930E04CDB7DEB7E8E00C941A
:10292000F72CE82FF0E0E657FA4FE185E03158F454
:10293000F894F0E0EE0FFF1FE55FFE4F208131813C
:102940007894C9010895E03121F0E13131F483E157
:1029500001C082E10E947A28089580E092E0089503
:10296000A2E2B0E0E6EBF4E10C94D12C9E012F5FE3
:102970003F4F80E1D9011D928A95E9F766ED71E03C
:1029800083EB95E029A33AA30E9424290E94940C8A
:102990001D8A1E8A1F8A188E312C212C00E0812C62
:1029A000912C540170E4472E71EE572E7DE9672E6D
:1029B00078E1772EE0E5CE2EE3ECDE2EE12CF12C53
:1029C00084EF91E0A0E0B0E08D8F9E8FAF8FB8A331
:1029D00080EC91EDA8E9BBE1898F9A8FAB8FBC8F1A
:1029E00080E491EEADE9B8E1898B9A8BAB8BBC8B1F
:1029F00083EB95E00E94382A892B09F4E1C083EB30
:102A000095E00E94652A9C0133272C32310509F498
:102A100042C0ACF42332310509F0ABC019821A82EE
:102A20001B821C821D821E821F82188619861A86AE
:102A30001B861C861D861E861F86188A60C024344D
:102A4000310529F02335310509F4B2C092C064E4A0
:102A500083EB95E00E94F6282AE030E040E451EE56
:102A60006DE978E183EB95E00E9484296CE283EBC9
:102A700095E00E94F6282AE030E040EC51ED68E94C
:102A80007BE183EB95E00E9484296CE283EB95E087
:102A90000E943629ADCF0F5F043009F0A9CF2981FC
:102AA0003A814B815C81A8EEB3E00E94592C698B7E
:102AB0007A8B8B8B9C8B2D813E814F8158850E9418
:102AC000592C698F7A8F8B8F9C8F29853A854B85FE
:102AD0005C852D8F3E8F4F8F58A32D853E854F856A
:102AE00058890E94592C6B017C0160323EE47307C7
:102AF0008105910530F462E38CE10E94B70A00E0A1
:102B000077CF603345E774078105910510F462E2E1
:102B1000F3CF60345CE975078105910510F466E236
:102B2000EBCF80E5C81683ECD806E104F10410F47D
:102B300062E1E2CF90E6C9169AEED906E104F1040B
:102B400010F465E1D9CFA0E7CA16A1E1DA06A1E049
:102B5000EA06F10410F461E0CFCFB0EACB16B6E894
:102B6000DB06B1E0EB06F10410F463E0C5CF65E0ED
:102B7000C3CF10ED180F1A3008F03ACFE1E0F0E0C3
:102B8000EC0FFD1F24E0029FE00DF11D11242081B8
:102B9000318142815381AAE0B0E00E94592C610F3B
:102BA000711D811D911D608371838283938320CF6A
:102BB00049885A886B887C88812C912C540118CFC5
:102BC00081149104A104B10489F4C301B2010E94EB
:102BD000260B61E070E080E090E00E945B271D8A98
:102BE0001E8A1F8A188E312C22242A948D8D9E8D48
:102BF000AF8DB8A188169906AA06BB06D0F40E942C
:102C0000E00A2D893E894F89588D280F311D411DBD
:102C1000511D2D8B3E8B4F8B588F381608F4382E54
:102C2000821508F4282E3FEF831A930AA30AB30AE9
:102C300056C0C301B20128EE33E040E050E00E94EC
:102C4000902CBA01A9012AE030E083EB95E00E94C4
:102C5000DB296CE283EB95E00E94F6284AE050E025
:102C6000632D83EB95E00E94EA296CE283EB95E00B
:102C70000E94F6286D897E898F89988DA50194011F
:102C80000E94902CBA01A9012AE030E083EB95E084
:102C90000E94DB296CE283EB95E00E94F6284AE073
:102CA00050E0622D83EB95E00E94EA296CE283EB11
:102CB00095E00E9436294C0C5D1C6E1C7F1C898D92
:102CC0009A8DAB8DBC8D84159505A605B70520F4AE
:102CD00049885A886B887C88812C912C54012989D9
:102CE0003A894B895C89283E33404105510509F0FA
:102CF0007FCEA296E2E10C94ED2CACE1B0E0E3E8EB
:102D0000F6E10C94DB2C0E9438276B017C0181E0FA
:102D10000E94960B14E703E0198361E0CE0101964F
:102D20000E94F30C0093A5050E94710C6AEF70E0FD
:102D300080E090E00E945B278091A505833089F4B4
:102D400083EB95E00E94382A892B59F40E9438279A
:102D50006C197D098E099F096038734C894C91402C
:102D6000D8F28091A505833009F44FC08FE70E9407
:102D70008F0A0E94A20A8983843511F083E05CC027
:102D80000E94A20A10921805809319050E94A20AB7
:102D90002091180530911905280F311D3093190520
:102DA000209318050E94A20A80931A050E94A20A85
:102DB00080931B05813110F7F12C0F2D10E08091CD
:102DC0001B0590E0880F991F0817190740F40E940F
:102DD000A20AF801E45EFA4F8083F394EECF80E715
:102DE000898361E0CE0101960E94F30C83E0809319
:102DF000A5050E94710C62E370E080E090E00E9403
:102E00005B278091A505833011F482E015C08FE720
:102E10000E948F0A0E94A20A8983803509F0AECFF2
:102E20000FE615E00E94A20AF80181938F01F5E0F8
:102E30000A381F07B9F781E06C96E8E00C94F72C8C
:102E400080911705992787FD9095A92FB92FFC012F
:102E50003196EB30F10508F066C0EC5CFF4F0C9446
:102E6000082D62E778E083EB95E00E94122984E761
:102E700093E00E94480D6AE578E083EB95E00E94BC
:102E8000122965E378E083EB95E00E9412296BE05C
:102E900078E083EB95E00E9412296AEE77E083EBFD
:102EA00095E00E9412296DEB77E083EB95E00E949C
:102EB000122967E977E083EB95E00E94122963E726
:102EC00077E083EB95E00E9412296CE477E083EBD6
:102ED00095E00E94122983EB95E00E94FE280E9453
:102EE000830D21C06FE277E01AC06AE077E017C077
:102EF00065EF76E014C066ED76E011C062E976E039
:102F00000EC06DE776E00BC068E676E083EB95E0F7
:102F10000E94122962E276E002C06CE076E083EB68
:102F200095E00E9412296AE070E080E090E00E9443
:102F30005B2783EB95E00E94382A892B29F083EBED
:102F400095E00E94652AF5CF0895ACE1B0E0EBEA88
:102F5000F7E10C94DB2C909117059F3F09F023C1FA
:102F6000482F50E0FA013A97EF36F10508F00FC10B
:102F7000E15CFF4F0C94082D63EE71E0A0C06FEE92
:102F800071E083EB95E00E94242985E789838BE13A
:102F9000EFE6F5E0DE01129601900D928A95E1F7D9
:102FA0006CE1CE0101960E94F30C0E94710C83E04B
:102FB0008093A50568EC70E080E090E00E945B27BC
:102FC0008091A505843009F0E2C08FE70E948F0A46
:102FD0000E94A20A8983853509F0D9C06DEE74E09C
:102FE00083EB95E00E9412296FEC74E083EB95E08F
:102FF0000E94122961EB74E096C067E072E083EBF7
:1030000095E00E94242989E6898361E0CE0101963A
:103010000E94F30C0E94710C83E08093A50568EC7C
:1030200070E080E090E00E945B278091A5058430ED
:1030300009F0ADC08FE70E948F0A0E94A20A89831F
:103040008E010E5F1F4F7E014DE1E40EF11C0E94C8
:10305000A20AF80181938F01EE15FF05C1F78BE1FC
:10306000FE013296AFE6B5E001900D928A95E1F748
:103070008981893409F08BC063E974E083EB95E0C2
:103080000E94122965E774E083EB95E00E94122903
:1030900067E574E048C061E272E083EB95E00E946E
:1030A00024298EEF8093170572C080528750805379
:1030B00090911A05981708F066C060E372E083EB00
:1030C00095E00E94242963C084E18093170560E2A3
:1030D00074E029C085E18093170569EE73E023C091
:1030E00086E18093170562EB73E01DC087E1809352
:1030F000170568E673E017C088E18093170567E558
:1031000073E011C089E18093170563E473E00BC09D
:103110008AE1809317056EE273E005C08BE180932E
:10312000170566E073E083EB95E00E9412292FC03B
:103130006CEE72E083EB95E00E94122980917D0590
:1031400091E01DC066ED72E083EB95E00E941229CC
:1031500080917D0592E013C061EC72E083EB95E015
:103160000E94122980917D0594E009C066EA72E010
:1031700083EB95E00E94122980917D0598E08927D4
:1031800080937D058FEF809317050E94241083EBB9
:1031900095E00E94382A892B09F45BC183EB95E006
:1031A0000E94652AF4CF0E942311882309F451C19B
:1031B0008091B104811104C08FEF8093170541C144
:1031C00040E050E060E070E082EB94E00E947F2DF0
:1031D00040911705042F112707FD1095212F312F3E
:1031E000F8013197EB31F10508F01BC1E255FF4FB3
:1031F0000C94082D552747FD509520911A0530E075
:10320000241735070CF40DC18B019C0101501109E5
:1032100021093109003211052105310558F0C0900E
:103220001B05EDE1F5E0F12CD12CA8E2EA2E41508E
:1032300051090FC0FA01E159FA4F61506083D9C0BA
:10324000DF0111972C9130E02417350729F0F39412
:103250003296FC10F5CFCBC00E2D10E020E030E010
:10326000061717072807390741F42081DA01A15909
:10327000BA4F11962C93DD24D394E394E8CF6F3F9B
:1032800071058105910511F008F0CBC060938705A9
:10329000B0C06F3F71058105910511F008F0C1C004
:1032A00060938805A6C06F3F71058105910511F0F7
:1032B00008F0B7C0609389059CC02091B2042062D9
:1032C0002037E9F440E050E060E070E083EB94E008
:1032D0000E947F2D9B01AC01DC01CB010197A1096C
:1032E000B1090897A105B10508F0AEC0A4EDB0E39F
:1032F0000E94592C6A5E7C4A8A46954E24C0263626
:10330000E9F440E050E060E070E083EB94E00E947C
:103310007F2D9B01AC01DC01CB010197A109B10913
:103320000797A105B10508F08FC0A8EAB1E60E9491
:10333000592C645E7C438E46944E05C06115710520
:103340008105910579F08B019C010054114E2D49A6
:1033500038410138F0EF1F07FAEF2F07F2E03F077F
:1033600008F05FC060937F057093800580938105AE
:10337000909382053EC06F3F71058105910511F064
:1033800008F04FC06093830534C08B019C0101504D
:103390001109210931090F3F11052105310508F0F7
:1033A00040C06093840525C08B019C01045C1940DA
:1033B000210931090D344DE114072105310528F4A7
:1033C000709386056093850514C0611571058105AC
:1033D000910521F48FEF80937E050BC06134710558
:1033E00081059105F0F4615060937E0502C0DD20F7
:1033F000C1F08091B00481111AC080914F05909165
:103400005005A0915105B09152050196A11DB11D25
:1034100080934F0590935005A0935105B0935205AA
:1034200006C062E472E083EB95E00E9424290E94CA
:1034300019118FEF809317056AE083EB95E00E94E6
:1034400036290E94241005C061E070E080E090E021
:103450007ACF6C96E8E00C94F72C6AE572E083EB87
:1034600095E00E94122962E472E083EB95E00E94ED
:10347000122983EB95E00E94382A892B31F083EBE7
:1034800095E00E94652A0E94A5170E947D16823051
:1034900029F0833051F46DE072E002C064E272E022
:1034A00083EB95E00E94122908958FEF8093170512
:1034B0001092B0040E942410809117058E3F69F08D
:1034C00083EB95E00E94382A892BB1F383EB95E0DA
:1034D0000E94652A0E94A517EFCF08950F931F93AE
:1034E000109117051F3F09F0D1C0893409F457C066
:1034F00000F5883309F468C058F4803309F476C0C5
:1035000008F060C08B3109F440C08132B1F1B8C01D
:10351000813409F486C030F4893309F465C08034FD
:1035200061F1AEC0823409F48DC0863409F447C01D
:10353000A7C0823609F486C078F4883531F128F4C2
:103540008235C1F18335E1F09BC08A3509F493C01F
:10355000813609F466C094C0823761F128F486365A
:1035600071F18936E1F08CC0883779F08A3709F437
:1035700082C0833709F084C003C063EE71E015C0D8
:103580000E94C30860E672E004C00E94CC086AE7AB
:1035900072E083EB95E00E9424298EEF6FC00E94B9
:1035A0009B070E940A0869E972E083EB95E00E949C
:1035B000242966C00E942A0862EB72E0F6CF0E94BE
:1035C000CE105EC080535AC06AEF71E083EB95E085
:1035D0000E94122990916E0588E0890F8871977E6C
:1035E000892B80936E051AC089E048C067EE71E0B0
:1035F00083EB95E00E94122980918F0590919005B0
:10360000A0919105B091920520E1822780938F05CA
:1036100090939005A0939105B09392051093170590
:103620002FC061ED71E083EB95E00E94122980913B
:103630008F0590919005A0919105B091920540E47D
:10364000842710C060EC71E083EB95E00E941229A2
:1036500080918F0590919005A0919105B091920570
:1036600020E2822780938F0590939005A093910587
:10367000B093920502C00E942D1A8FEF8093170518
:10368000809117058E3F09F0D4C0DDC00E94231140
:10369000882309F4D8C08091B104811104C08FEF50
:1036A00080931705C6C040E050E060E070E082EB18
:1036B00094E00E947F2D00911705112707FD1095BA
:1036C000212F312FF8013197E930F10508F0B4C00E
:1036D000E753FF4F0C94082D8B019C010154114EB0
:1036E0002D4938410F37104F2A4F324008F0A4C0FF
:1036F00060934B0570934C0580934D0590934E0558
:1037000077C060934F057093500580935105909357
:10371000520581E08093B0046BC06830710581056B
:10372000910508F089C06093530562C08B019C012C
:1037300001501109210931090A301105210531050E
:1037400008F07AC06093540553C061EB71E082EBDE
:1037500094E00E94B92E10E0009799F00E94932EF9
:10376000009779F0183130F4E12FF0E0EA5BFA4F7E
:1037700087871F5F61EB71E080E090E00E94B92EC7
:10378000EBCF1831A8F5E12FF0E0EA5BFA4F17868E
:103790001F5FF7CF653071058105910508F04CC0BA
:1037A00060936D0525C08B019C0101501109210911
:1037B00031090630110521053105F0F520916E051E
:1037C000287F262B20936E0513C08B019C0101508E
:1037D0001109210931090115124C2140310560F50B
:1037E00060934705709348058093490590934A0577
:1037F0008091B004811113C080914F0590915005C4
:10380000A0915105B09152050196A11DB11D809363
:103810004F0590935005A0935105B09352050E9417
:1038200019118FEF809317056AE083EB95E00E94F2
:1038300036290E94201707C062E472E083EB95E00E
:103840000E942429ECCF1F910F9108958FEF809350
:1038500017051092B0040E942017809117058E3F23
:1038600069F083EB95E00E94382A892BB1F383EB52
:1038700095E00E94652A0E946E1AEFCF6AE070E020
:1038800080E090E00E945B2783EB95E00E94382A5D
:10389000892B29F083EB95E00E94652AF5CF0895E6
:1038A000CF93C82F682F83EB95E00E94922A9091C6
:1038B0003C059C2790933C05CF910895A1E0B0E092
:1038C000E4E6FCE10C94E12C99830E94501C998160
:1038D000892F0E94501C2196E2E00C94FD2C1F932E
:1038E000CF93DF93182FEB0110923C0565EB70E04E
:1038F00083EB95E00E94590662E670E083EB95E069
:103900000E945906812F0E94501CCE010E945E1C0D
:10391000DF91CF911F91089560913C0583EB95E075
:103920000E94922A0895A1E2B0E0E9E9FCE10C943A
:10393000DD2C7B018A018B3009F42DC108F03FC0DA
:10394000853009F49BC010F5823009F47EC058F42C
:10395000813009F02FC269E270E081E00E946F1CA3
:1039600006E415E068C0833009F480C0843009F0B3
:1039700021C261E070E084E00E946F1C81E00E943F
:10398000501C0E948C1C0E94B0141EC2883009F486
:103990009BC070F4863009F48DC0873009F00AC2EC
:1039A00061E070E087E00E946F1C80911A0508C2F8
:1039B000893009F491C08A3009F4C3C0FBC189364B
:1039C00009F468C178F4863609F419C120F4853603
:1039D00009F401C1EFC1873609F425C1883609F41D
:1039E0002AC1E8C18C3609F49EC190F48A3609F4E4
:1039F0005BC18B3609F0DEC161E070E08BE60E94AE
:103A00006F1CF80180810E94F2070E94CC08BDC1A2
:103A10008D3609F4BCC1873C09F0CCC161E070E08F
:103A200087EC0E946F1C81E00E94501C0E948C1C3D
:103A300010923D05C9C1F80181918F010E94501C6F
:103A4000F5E00F361F07B9F7BDC16BE170E082E00A
:103A50000E946F1C0FE615E0F80181918F010E9412
:103A6000501CF5E00A381F07B9F7ACC161E070E0FF
:103A700083E00E946F1C0E947D16A2C160911B050D
:103A800070E0660F771F85E00E946F1C0CE115E067
:103A900080911B0590E0880F991F98012C513540AB
:103AA0002817390708F08EC1F80181918F010E9413
:103AB000501CEECF62E070E086E00E946F1C84E74D
:103AC00093E00E945E1C7EC161E070E088E00E948D
:103AD0006F1C8091A30574C186E6898361E0CE01E5
:103AE00001960E94F30C0E94710C83E08093A5055F
:103AF00068EC70E080E090E00E945B278091A50573
:103B00008430D9F48FE70E948F0A0E94A20A898329
:103B1000863469F460E270E089E00E946F1C10E274
:103B20000E94A20A0E94501C1150D1F74BC161E0C3
:103B300070E089E00E946F1C28C161E070E089E0BC
:103B40003CC169E170E08AE00E946F1C10928A0516
:103B50002091A40580918F0590919005A0919105E9
:103B6000B0919205222311F0806801C08F77809375
:103B70008F0590939005A0939105B09392050AE864
:103B800015E0F80181918F010E94501CF5E0033A85
:103B90001F07B9F717C161E270E08BE00E946F1C4C
:103BA00080917C048F3F39F080917C0491E0980FE4
:103BB00090937C0402C080917C040E94501C10E011
:103BC000812F0E9491140E94210A0E945E1C1F5F97
:103BD0001031B1F7F7C061E070E085E60E946F1C1C
:103BE00089E2E816F10409F0EAC0D801E6E4F5E05C
:103BF0008D91819385E0EF36F807D1F7C6C061E07B
:103C000070E086E60E946F1CEBE1EE16F10409F00D
:103C1000D6C0D801EFE6F5E08D91819385E0EA38D2
:103C2000F807D1F7B2C061E070E087E60E946F1C30
:103C30000E94C308AAC061E070E088E60E946F1C81
:103C400085E789838BE1EFE6F5E0DE0112960190CE
:103C50000D928A95E1F76CE1CE0101960E94F30C7A
:103C60000E94710C83E08093A50560E273E080E020
:103C700090E00E945B278091A505843009F09FC0E9
:103C80008FE70E948F0A0E94A20A8983853509F076
:103C900096C07BC061E070E089E60E946F1C0E94C4
:103CA0009B070E940A0871C061E070E08AE60E94EA
:103CB0006F1C89E6898361E0CE0101960E94F30CB6
:103CC0000E94710C83E08093A50560E273E080E0C0
:103CD00090E00E945B278091A505843009F06FC0B9
:103CE0008FE70E948F0A0E94A20A89838E010E5FCD
:103CF0001F4F7E01EDE1EE0EF11C0E94A20AF801B9
:103D000081938F01EE15FF05C1F78BE1FE0132961D
:103D1000AFE6B5E001900D928A95E1F7898189348B
:103D200009F04DC032C061E070E08CE60E946F1C6B
:103D3000F0E2EF16F10461F487E6898380E2F8018E
:103D4000DE01129601900D928A95E1F761E203C0BF
:103D500087E4898361E0CE0101960E94F30C0E9402
:103D6000710C83E08093A5056CE474E080E090E042
:103D70000E945B278091A505843009F58FE70E949A
:103D80008F0A0E94A20A8734D1F481E019C061E051
:103D900070E08DE60E946F1C89E1E816F10479F469
:103DA000D801EAE8F5E08D91819385E0E33AF807E0
:103DB000D1F7EBCF61E070E08AEC0E946F1C80E0ED
:103DC0000E94501C0E948C1CA196E6E00C94F92CD9
:103DD000A0E0B0E0EEEEFEE10C94DB2CCCE9D3E009
:103DE00014E606E035E0F32E44E0E42E53E0D52E51
:103DF00062E0C62E83EB95E00E94382A892B09F4F5
:103E00009BC083EB95E00E94652A282F80930704CE
:103E10004091060450E04730510560F7FA01EE5238
:103E2000FF4F0C94082D853B29F781E08093060411
:103E3000E1CF823609F07DC0C0920604DBCF8093CB
:103E4000050480930404D0920604D4CF9C01332748
:103E500030930304209302049091040498279093D4
:103E60000404E0920604C6CF382F222740910204B2
:103E700050910304242B352B309303042093020428
:103E800090910404982790930404F0920604253638
:103E9000310508F4AFCF61E070E08CEC0E946F1C3C
:103EA00081E00E94501C0E948C1C43C020910004A1
:103EB00030910104F901E456FC4F80839091040491
:103EC000982790930404C90101969093010480936C
:103ED000000420910204309103048217930708F430
:103EE00089CF0093060486CF8091040482130BC00F
:103EF00060910004709101044CE953E08091050445
:103F00000E94931C0DC062E070E08BEC0E946F1C5D
:103F1000809105040E94501C80913C050E94501C19
:103F2000FE01812F11928A95E9F7109201041092F7
:103F30000004109206045ECFCDB7DEB7E8E00C9423
:103F4000F72C81E080933D0580913D05882349F061
:103F500083EB95E00E94382A892BB1F30E94E81E7A
:103F6000F3CF0895AAE2B0E0E8EBFFE10C94D92C7E
:103F70000E942C276B017C0181E00E94960B83EB51
:103F800095E00E94382A892B29F083EB95E00E9466
:103F9000652AF5CF5E98409811E072E6B72EE9E207
:103FA000AE2E03E00E942C276C197D098E099F0913
:103FB000693C710581059105E0F11123D1F10E9461
:103FC0002C276B017C015D9A419A80ED97E00E945D
:103FD0006A06B982E6E4F5E0DE0112968A2D0190C8
:103FE0000D928A95E1F76AE2CE0101960E94F30CE8
:103FF0005D98419880E090E00E946A060093A505D4
:104000000E94710C62E370E080E090E00E945B2708
:104010008091A505843061F40093A5058FE70E9487
:104020008F0A0E94A20A11E0823419F410E001C044
:1040300011E083E10E945128892BA1F411E012C004
:104040005E9A409A5D9A419A83EB95E00E94652AB8
:104050008D309105B9F06CF40A97A1F05E98409804
:104060005D98419883EB95E00E94382A892B41F7AF
:1040700099CF8332910579F08234910579F70E94C6
:10408000A11FECCF62EB71E083EB95E00E94122957
:104090000E94261CE3CF0E94B014E0CF8F929F9223
:1040A000AF92BF92CF92DF92EF92FF921F93CF9386
:1040B000DF9383E10E945128892B09F078C068ECD6
:1040C00070E080E090E00E945B2780E090E00E943A
:1040D0006A060E942C274B015C016B017C0180EC7D
:1040E000C80E82E1D81EE11CF11C0E942C276C1521
:1040F0007D058E059F0530F483E10E945128892BB0
:10410000A1F353C083E10E945128892B09F04DC0CF
:1041100080ED97E00E946A060E942C276B017C01CB
:10412000D0E0C1E088E4880E86E2981EA11CB11C94
:1041300011E083E10E945128892B21F58C149D0404
:10414000AE04BF0430F480ED97E00E946A06D1E02F
:10415000F0CF0E942C276C197D098E099F09693CBC
:1041600071058105910528F30E942C276B017C01C4
:10417000C12719F080ED97E002C080E090E00E9436
:104180006A06D7CF80E090E00E946A06DD2349F0FE
:104190008091A3058F5F83700E94F2070E94CC0874
:1041A00006C00E942A080E94C3080E94B21FDF9125
:1041B000CF911F91FF90EF90DF90CF90BF90AF9085
:1041C0009F908F900895CF92DF92EF92FF9280E0C0
:1041D0000E949C060E94730661E086E00E94E5272B
:1041E00061E085E00E94E52761E08EE00E94E5271E
:1041F00061E08FE00E94E52760E083E10E94E5270F
:1042000060E088E00E94E52761E088E00E941E28C7
:104210000E94610640E052EC61E070E083EB95E0C3
:104220000E94802B0E94E5070E94CC080E94741215
:104230008FEF80937C040E94880678940E942C273C
:104240006B017C0180917C048F3F59F40E942C27E4
:104250006C197D098E099F09603D774081059105A4
:1042600088F380ED97E00E946A0661E083E10E9496
:104270001E285E9A409A83EB95E00E94382A892B8B
:1042800029F083EB95E00E94652AF5CF6FEC72E090
:1042900083EB95E00E94F32884E793E00E94480DA9
:1042A00066EE72E083EB95E00E94F3284AE050E06E
:1042B00067E070E083EB95E00E94C32962E370E061
:1042C00080E090E00E945B2783EB95E00E94382A13
:1042D00004970CF183EB95E00E94652A82349105E6
:1042E000D1F483EB95E00E94652A8E34910599F410
:1042F00083EB95E00E94652A8434910561F483EB99
:1043000095E00E94652A819731F480E090E00E9458
:104310006A060E94B21F409147055091480560917E
:10432000490570914A05DB01CA010197A109B1094C
:104330000497A105B10568F440937B04433029F448
:1043400040EA56E861E070E004C040E052EC61E011
:1043500070E083EB95E00E94802B0E944E205E98D7
:10436000409880E090E00E946A060E9474121092C9
:10437000970480918F0583FF11C080915B0588238E
:1043800051F080916205882331F08091690588237E
:1043900011F087E001C085E08093970480E00E94DF
:1043A000960B809198040E94CA0A0E94710C109288
:1043B00011041092100410920F04F12C8091A305A7
:1043C0008F15B0F062E370E080E090E00E945B2720
:1043D00080ED97E00E946A0662E370E080E090E082
:1043E0000E945B2780E090E00E946A06F394E6CF8B
:1043F00080916E0584FF08C0982F987181E09831F4
:1044000009F080E00E9491118FE00E949C06FF90CD
:10441000EF90DF90CF900895EF92FF920F931F934C
:10442000CF93DF938C016EE770E083EB95E00E9401
:104430005906E801F12CF0E2EF2E8E0188818D57AC
:10444000823048F46DE770E083EB95E00E945906F6
:1044500088818E2588832196F801608183EB95E021
:104460000E94922AF394F9E0FF12E7CF6EE770E022
:1044700083EB95E00E945906CDB7DEB7E6E00C94D9
:10448000F92CA9E0B0E0E7E4F2E20C94E12C909181
:10449000990491110EC09EEF99838A836B8350E03B
:1044A000559547954C832D83198618861F821E8249
:1044B0002EC040919E04842F90E0B4E0959587959E
:1044C000BA95E1F7242F2F7030E08217930719F186
:1044D0008DEF89831B82FE01349650E0842F90E09B
:1044E000A4E095958795AA95E1F7242F2F7030E0E9
:1044F0008217930749F0DC01A156BB4F8C91819341
:10450000405F5F5F563051F740939E045A83CE015F
:1045100001960E940C228091990490E0019666E039
:1045200070E00E947C2C809399042996E2E00C9420
:10453000FD2CA0E0B0E0EFE9F2E20C94DA2C6C0183
:104540006EE770E083EB95E00E9459068601E12C4E
:10455000F12CC0E0D0E030E2B32EF801608183E8B6
:10456000860F823078F46DE770E083EB95E00E946F
:104570005906F80160816B2570E083EB95E00E949D
:10458000590604C083EB95E00E94922AE114F104DD
:1045900059F0F80180819E01280F311DC901C92FF2
:1045A000DD27C80FD91FDD273FEFE31AF30A89E0A3
:1045B000E816F10459F028E0E216F10421F48C2FFA
:1045C0008095F60180870F5F1F4FC7CFCDB7DEB74D
:1045D000E9E00C94F62CA9E0B0E0E1EFF2E20C94F3
:1045E000E12CE82F362F8091990490E0019664E247
:1045F00070E00E947C2C8093990458E9598350E123
:104600005A83813089F048F08230B9F08330D9F490
:104610008B8381EF8C833D8319C085E08B8381EF91
:104620008C832F5F2D8312C08B8381EF8C8384E674
:10463000489FA00111245D8309C084E08B8381EF32
:104640008C83ED8303C00E94CE1104C0CE0101967D
:104650000E9499222996E2E00C94FD2CA2E0B0E0A1
:10466000E4E3F3E20C94D62C182F762E2A834983A8
:104670000E9438276B017C018091AF0480909A04DE
:1046800090909B04A0909C04B0909D042A81498145
:104690008823C1F0D701C60188199909AA09BB0965
:1046A0004C015D0191EE89169EE29906A104B104C8
:1046B00020F1241708F4422F202F672D812F0E940C
:1046C000EB2213C0D701C60188199909AA09BB09B1
:1046D0004C015D0191E3891695E79906A104B104A7
:1046E00060F0672D812F0E944122C0929A04D092DF
:1046F0009B04E0929C04F0929D042296EDE00C94C1
:10470000F22CA2E2B0E0E7E8F3E20C94D72C8CE0C4
:104710000E94B10A81110FC06EEE72E083EB95E04A
:104720000E9424295E9A409A80E00E94960B0E9483
:10473000710C5E98409883EB95E00E94382A892B93
:1047400001F183EB95E00E94652A90917B04992307
:1047500019F00E949912EFCF4091100450E09A0195
:104760002F5F3F4F2F7133276091110470E02617A0
:10477000370709F3FA01E55EFB4F808320931004AD
:10478000DACF8091A505843009F086C00E943827D1
:10479000611571058105910549F060938904709355
:1047A0008A0480938B0490938C040CC081E090E089
:1047B000A0E0B0E08093890490938A04A0938B04D6
:1047C000B0938C0480917F049091800481609093D9
:1047D000800480937F0483E08093A5058FE70E9487
:1047E0008F0A0BE314E00E94A20AF80181938F0163
:1047F000F4E004341F07B9F72091440480913B048E
:10480000982F922796FF3BC090E492279093440400
:10481000982F98739833F1F410E0212F30E08091B5
:104820003B04877090E0821793074CF11F5F209143
:104830006E05812F90E0FC01E55CFB4F24FF04C076
:1048400080810E94B011E9CF608183EB95E00E94E6
:10485000922AE3CF8F7399F480913C04809388046B
:1048600080913D048093860480913E04809385046A
:104870008091410490E090937E0480937D04809128
:104880000F04813019F482E080930F0480910F04AB
:10489000833011F410920F040E9438276B017C01C1
:1048A0008091810490918204A0918304B09184044A
:1048B0000097A105B105C9F0A7019601281B390B86
:1048C0004A0B5B0BDA01C901883B9B40A105B1058E
:1048D00060F00E94E00A8093870410928104109295
:1048E0008204109283041092840480918D0490912C
:1048F0008E04A0918F04B091900446015701881A4C
:10490000990AAA0ABB0A86E495E00E940C09861659
:104910009706A806B90608F4A5C0C0928D04D092E7
:104920008E04E0928F04F09290040E9457068091CA
:104930007C048830A0F080918F0590919005A09123
:104940009105B09192056CE1B695A79597958795DD
:104950006A95D1F7892B8A2B8B2B09F0ABC18091FB
:104960007C048F5F80937C048091890490918A04F9
:10497000A0918B04B0918C040097A105B105F1F0D2
:10498000C81AD90AEA0AFB0A86E495E00E940C09D3
:104990006C157D058E059F0508F004C180918F057B
:1049A00084FD04C080ED97E00E946A06109289049D
:1049B00010928A0410928B0410928C0490914404FB
:1049C000907C9093440450911004809111042091A4
:1049D0000F04581709F403C1223009F000C19058A0
:1049E00090934404E0916E05E770F0E0E45BFC4FC7
:1049F0006081693008F0DBC0615040E04613D9C0E7
:104A00008093110487E3840F90914404892B809351
:104A100044044093120483E080930F045D9A419A0A
:104A200090919704911130C1809198040E94CA0A14
:104A3000E0916E05E770F0E0E45BFC4F608184E498
:104A400094E00E94AC0CE0919804EF5FE09398042E
:104A5000E83109F42CC1F0E0EA5BFA4F878588233E
:104A600009F425C10E941B0D813069F580916E0506
:104A7000887149F180917F0490918004880F991F7B
:104A80009093800480937F0483E08093A5050E9427
:104A9000710C0E9438276093810470938204809384
:104AA000830490938404672B682B692B61F481E065
:104AB00090E0A0E0B0E08093810490938204A09302
:104AC0008304B093840480916E0584FF1FC080919D
:104AD0007F04909180048E7F0E94420A182F60917B
:104AE0007D04809188040E948F12482F612F80914D
:104AF000870449A30E948F120091A305282F49A182
:104B000060918504809186040E942E235D984198CF
:104B1000809195048130C1F018F08230B1F1D4C099
:104B200083E10E945128892B09F0CEC081E0809357
:104B300095040E942C2760939104709392048093B3
:104B4000930490939404C0C083E10E945128892B60
:104B500031F50E942C27C0909104D0909204E090EF
:104B60009304F09094046C197D098E099F09693EA5
:104B700073408105910508F4A7C082E080939504F5
:104B800080ED97E00E946A069FC083E10E94512851
:104B9000892B09F499C080E090E00E946A06109287
:104BA000950492C080E090E00E946A0607CF68E01A
:104BB00024CF851709F424CF4F5F242F30E090E0F5
:104BC000F901EC5BFB4FDC01A55EBB4F7C91708370
:104BD000F901EE5EFB4F708301968F710FCF243089
:104BE000B1F42091120483E194E0A5E4B4E0FC0167
:104BF0003E2F381B321718F431913D93F9CF87E3DC
:104C0000820F90914404892B8093440404CF8091B7
:104C10009504823071F49160909344045E9A409AB6
:104C200053E9E52E55E0F52E8E010F5F1F4FB801B9
:104C300011C05E98409880910F04811103C081E0FB
:104C400080930F0480910F04833051F784E08093A8
:104C50000F04E6CFF70181917F0169A37AA30E9437
:104C60009114F801819391938F0169A17AA1F3EADC
:104C7000EF16F5E0FF0671F780916E0545E454E00C
:104C800087700E949109CACE80915305882309F448
:104C9000CBCE2091960431E0320F30939604291345
:104CA00003C01092960481500E94910BBDCE1092C9
:104CB0009804D8CE80917C04883011F45E9A409A92
:104CC00089E080937C04CECEA296ECE00C94F32C89
:104CD0008230E8F4E82FF0E0EE0FFF1FEA55FA4FBC
:104CE00071836083813041F0809169008C7F842BD7
:104CF00080936900E89A089580916900440F551FD8
:104D0000440F551F837F842B80936900E99A08958F
:104D10001F920F920FB60F9211242F933F934F9330
:104D20005F936F937F938F939F93AF93BF93EF9313
:104D3000FF938091A6059091A705892B29F0E0911A
:104D4000A605F091A7050995FF91EF91BF91AF914D
:104D50009F918F917F916F915F914F913F912F9193
:104D60000F900FBE0F901F9018951F920F920FB6C5
:104D70000F9211242F933F934F935F936F937F93E1
:104D80008F939F93AF93BF93EF93FF938091A80569
:104D90009091A905892B29F0E091A805F091A9052A
:104DA0000995FF91EF91BF91AF919F918F917F9165
:104DB0006F915F914F913F912F910F900FBE0F9088
:104DC0001F9018951F920F920FB60F9211242F93D8
:104DD0003F938F939F93AF93BF938091AB05909137
:104DE000AC05A091AD05B091AE053091AA0523E0C8
:104DF000230F2D3720F40196A11DB11D05C026E813
:104E0000230F0296A11DB11D2093AA058093AB0527
:104E10009093AC05A093AD05B093AE058091AF051E
:104E20009091B005A091B105B091B2050196A11D78
:104E3000B11D8093AF059093B005A093B105B093D9
:104E4000B205BF91AF919F918F913F912F910F909C
:104E50000FBE0F901F9018952FB7F8946091AB0577
:104E60007091AC058091AD059091AE052FBF08956E
:104E70003FB7F8948091AF059091B005A091B1052E
:104E8000B091B20526B5A89B05C02F3F19F0019639
:104E9000A11DB11D3FBF6627782F892F9A2F620F62
:104EA000711D811D911D42E0660F771F881F991F9C
:104EB0004A95D1F70895CF92DF92EF92FF92CF9368
:104EC000DF936B017C010E943827EB01C114D104F0
:104ED000E104F10479F00E9438276C1B7D0B683ED9
:104EE0007340A0F381E0C81AD108E108F108C85165
:104EF000DC4FECCFDF91CF91FF90EF90DF90CF9020
:104F00000895789484B5826084BD84B5816084BD41
:104F100085B5826085BD85B5816085BDEEE6F0E032
:104F2000808181608083E1E8F0E01082808182608E
:104F30008083808181608083E0E8F0E0808181600F
:104F40008083E1EBF0E0808184608083E0EBF0E03F
:104F5000808181608083EAE7F0E0808184608083E3
:104F6000808182608083808181608083808180688D
:104F700080831092C1000895833081F028F481303D
:104F800099F08230A1F008958630A9F08730B9F009
:104F90008430D1F4809180008F7D03C080918000A7
:104FA0008F7780938000089584B58F7702C084B591
:104FB0008F7D84BD08958091B0008F7703C080916C
:104FC000B0008F7D8093B0000895CF93DF9390E081
:104FD000FC01ED50F44F2491FC01E95FF34F849103
:104FE000882349F190E0880F991FFC01E15DF34FA0
:104FF000A591B4918B5D934FFC01C591D4919FB75E
:10500000611108C0F8948C91209582238C9388813B
:1050100082230AC0623051F4F8948C91322F30957B
:1050200083238C938881822B888304C0F8948C918D
:10503000822B8C939FBFDF91CF910895A1E0B0E0C8
:10504000E4E2F8E20C94DF2C282F30E0F901E15281
:10505000F44F8491F901ED50F44F1491F901E95F97
:10506000F34F04910023C9F0882321F069830E9443
:10507000BC276981E02FF0E0EE0FFF1FEB5DF34FDF
:10508000A591B4919FB7F8948C91611103C01095CC
:10509000812301C0812B8C939FBF2196E4E00C9467
:1050A000FB2CCF93DF93282F30E0F901E152F44F2E
:1050B0008491F901ED50F44FD491F901E95FF34F78
:1050C000C491CC2391F081110E94BC27EC2FF0E019
:1050D000EE0FFF1FE55EF34FA591B4912C912D23A8
:1050E00081E090E021F480E002C080E090E0DF9178
:1050F000CF9108958E3008F08E50877020919D01D9
:1051000090E4299F90011124822B80937C00809150
:105110007A00806480937A0080917A0086FDFCCFCB
:10512000809178002091790090E0922B0895A0E082
:10513000B0E0EDE9F8E20C94DB2C6C017A01EB01B4
:10514000E60EF71E00E010E0CE15DF0561F0699174
:10515000D601ED91FC910190F081E02DC6010995F9
:10516000080F191FF1CFC801CDB7DEB7E8E00C94E6
:10517000F72C6115710589F0DB010D900020E9F72E
:10518000AD0141505109461B570BDC01ED91FC91DB
:105190000280F381E02D0995089580E090E0089564
:1051A000EF92FF920F931F93CF93DF938C01FB013C
:1051B000C0E0D0E064917F018FEFE81AF80A66231F
:1051C00061F0D801ED91FC910190F081E02DC801D2
:1051D0000995C80FD91FF701EDCFCE01CDB7DEB7C6
:1051E000E6E00C94F92C0E94B9280895DC01ED91B9
:1051F000FC910190F081E02D099508950F931F9384
:10520000CF93DF93EC016DE00E94F6288C016AE0F9
:10521000CE010E94F628800F911FDF91CF911F9140
:105220000F9108950F931F93CF93DF93EC010E948A
:10523000D0288C01CE010E94FE28800F911FDF91A3
:10524000CF911F910F9108950F931F93CF93DF93E9
:10525000EC010E94B9288C01CE010E94FE28800F2B
:10526000911FDF91CF911F910F9108950F931F937D
:10527000CF93DF93EC010E94F6288C01CE010E94AF
:10528000FE28800F911FDF91CF911F910F910895FC
:10529000A1E2B0E0EEE4F9E20C94D72C7C01C42E3C
:1052A000E52FCB01D22E19A221E02D1510F02AE016
:1052B000D22E8E010F5D1F4F8D2C912CA12CB12C65
:1052C0006C2D7E2FA50194010E94902C8C2DD29ED6
:1052D00080191124015011098A3010F4805D01C039
:1052E000895CF8018083211531054105510521F0C4
:1052F000C22EE32FCA01E4CFB801C7010E94B9282A
:10530000A196ECE00C94F32CA0E0B0E0EAE8F9E21E
:105310000C94DB2CEC016A017B012115310541F471
:10532000E881F9810190F081E02D642F09951DC07D
:105330002A303105A9F477FF12C06DE20E94F628E9
:105340008C0144275527BA014C195D096E097F0964
:105350002AE0CE010E944829800F911F06C02AE052
:10536000B701A601CE010E944829CDB7DEB7E8E01B
:105370000C94F72C9A01AB01662757FD6095762FA8
:105380000E94842908950F931F93CF93DF93EC011C
:105390009A01AB01662757FD6095762F0E948429FC
:1053A0008C01CE010E94FE28800F911FDF91CF91CA
:1053B0001F910F9108952115310549F4DC01ED91FC
:1053C000FC910190F081E02D642F099508950E94D1
:1053D000482908959A01462F50E060E070E00E944D
:1053E000DB2908959A01AB0160E070E00E94DB299F
:1053F00008950F931F93CF93DF93EC010E94DB2955
:105400008C01CE010E94FE28800F911FDF91CF9169
:105410001F910F9108950F931F93CF93DF93EC018A
:105420009A01AB0160E070E00E94DB298C01CE01A3
:105430000E94FE28800F911FDF91CF911F910F9145
:1054400008950F931F93CF93DF93EC019A01462F9A
:1054500050E060E070E00E94DB298C01CE010E94E8
:10546000FE28800F911FDF91CF911F910F9108951A
:10547000FC0124853585F901E05CFF4F8081918135
:10548000F901EE5BFF4F20813181821B930B8F73FB
:1054900099270895FC0184859585FC01E05CFF4F08
:1054A00040815181FC01EE5BFF4F20813181421729
:1054B000530741F00190F081E02DE80FF91F808142
:1054C00090E008958FEF9FEF0895FC018485958506
:1054D000FC01E05CFF4F40815181FC01EE5BFF4F1E
:1054E000208131814217530779F0A081B181A80F43
:1054F000B91F8C91208131812F5F3F4F2F7333274C
:105500003183208390E008958FEF9FEF0895FC0191
:1055100081A1882329F0A489B5898C9186FFFBCFCE
:1055200011A20895CF93DF93FC0126853785D90119
:10553000A05CBF4F8D919C91119701968F73992715
:10554000E901CE5BDF4F4881598184179507D9F374
:105550000D90BC91A02DA20FB31F6C93A685B785AB
:10556000A05CBF4F11969C938E93A689B7892C910E
:1055700081E090E0078C02C0880F991F0A94E2F73F
:10558000282B2C9381E081A30488F589E02D80816C
:105590008064808381E090E0DF91CF910895089549
:1055A0001F920F920FB60F9211242F933F934F9398
:1055B0008F939F93EF93FF938091C00082FD1CC057
:1055C0004091C6008091590690915A0601968F73BA
:1055D000992720915B0630915C068217930771F042
:1055E000E0915906F0915A06E75EF94F4083909397
:1055F0005A068093590602C08091C600FF91EF9130
:105600009F918F914F913F912F910F900FBE0F90CF
:105610001F90189583EB95E00E94382A892B11F092
:105620000E94CF2A08951F920F920FB60F92112455
:105630002F933F938F939F93EF93FF9320911506A2
:105640003091160680911706909118062817390791
:1056500031F48091C1008F7D8093C10014C0E0912E
:105660001706F0911806EB52FA4F20818091170629
:105670009091180601968F7399279093180680933E
:1056800017062093C600FF91EF919F918F913F9154
:105690002F910F900FBE0F901F901895A0E0B0E0D3
:1056A000E4E5FBE20C94D72CFC011382128288EE15
:1056B00093E0A0E0B0E084839583A683B7838EE86F
:1056C00093E0918380837587648757874687318B02
:1056D000208B138B028BF58AE48AD78AC68AB18E17
:1056E000A08E938E828E8F85848F8889858F8989FD
:1056F000868F8A89878F8B8980A3ECE00C94F32CAA
:10570000CF92DF92EF92FF92CF93DF93EC016A0189
:105710007B01411581EE580761057105F9F0EC89AF
:10572000FD8981E090E008A002C0880F991F0A94CB
:10573000E2F7808360E079E08DE390E0A7019601D5
:105740000E94902C215031094109510956954795E5
:1057500037952795211580E1380798F0EC89FD8968
:10576000108260E874E88EE190E0A70196010E9443
:10577000902C21503109410951095695479537958B
:105780002795E889F9893083EA89FB89208319A262
:10579000EE89FF89408181E090E09C010C8C02C081
:1057A000220F331F0A94E2F7422B4083EE89FF89D0
:1057B00040819C010D8C02C0220F331F0A94E2F736
:1057C000422B4083EE89FF8940819C010E8C02C0F0
:1057D000220F331F0A94E2F7422B4083EE89FF89A0
:1057E00020810F8C02C0880F991F0A94E2F78095E0
:1057F00082238083DF91CF91FF90EF90DF90CF9055
:1058000008958F929F92AF92BF92CF92DF92EF92C4
:10581000FF920F931F9381E08F9385E08F9387E032
:105820008F9383E08F9384E08F93E6EC8E2E912C00
:10583000F2ECAF2EB12CA1ECCA2ED12CB0ECEB2E99
:10584000F12C04EC10E025EC30E045ED55E069E189
:1058500076E083EB95E00E944E2B0F900F900F9017
:105860000F900F901F910F91FF90EF90DF90CF90CE
:10587000BF90AF909F908F9008950E9481270E94C3
:10588000E320CAE0DBE20E9481232097E1F30E943B
:105890000A2BF9CFA29FB001B39FC001A39F700D47
:1058A000811D1124911DB29F700D811D1124911D28
:1058B00008950E944A2CA59F900DB49F900DA49F1F
:1058C000800D911D11240895B7FF0C94592C0E944E
:1058D000592C821B930B0895DB018F939F930E9499
:1058E000592CBF91AF91A29F800D911DA39F900D48
:1058F000B29F900D1124089597FB072E16F4009483
:1059000007D077FD09D00E940E2D07FC05D03EF48C
:10591000909581959F4F0895709561957F4F08955B
:10592000A1E21A2EAA1BBB1BFD010DC0AA1FBB1FA3
:10593000EE1FFF1FA217B307E407F50720F0A21B15
:10594000B30BE40BF50B661F771F881F991F1A9482
:1059500069F760957095809590959B01AC01BD01AC
:10596000CF010895052E97FB1EF400940E94C92CC8
:1059700057FD07D00E94902C07FC03D04EF40C94E6
:10598000C92C50954095309521953F4F4F4F5F4F13
:10599000089590958095709561957F4F8F4F9F4F9B
:1059A00008952F923F924F925F926F927F928F92C3
:1059B0009F92AF92BF92CF92DF92EF92FF920F939E
:1059C0001F93CF93DF93CDB7DEB7CA1BDB0B0FB6A8
:1059D000F894DEBF0FBECDBF09942A883988488865
:1059E0005F846E847D848C849B84AA84B984C884FB
:1059F000DF80EE80FD800C811B81AA81B981CE0FF2
:105A0000D11D0FB6F894DEBF0FBECDBFED010895D6
:105A1000EE0FFF1F0590F491E02D0994AA1BBB1B0C
:105A200051E107C0AA1FBB1FA617B70710F0A61B9E
:105A3000B70B881F991F5A95A9F780959095BC01BF
:105A4000CD0108958F929F92AF92BF92CF92DF9235
:105A5000EF92FF92CF93DF93EC01688179818A8185
:105A60009B81611571058105910521F464E279ED51
:105A70008BE597E02DE133EF41E050E00E94B22C3E
:105A800049015A019B01AC01A7EAB1E40E94592CDB
:105A90006B017C01ACEEB4EFA50194010E94672C70
:105AA000C60ED71EE81EF91EF7FE06C081E0C81A12
:105AB000D108E10880E8F80AC882D982EA82FB822C
:105AC000C701B6019F77DF91CF91FF90EF90DF90F4
:105AD000CF90BF90AF909F908F9008950E94222DFD
:105AE000089586E091E00E94222D089560930601BA
:105AF00070930701809308019093090108952F92F4
:105B00003F925F926F927F928F929F92AF92BF92DD
:105B1000CF92DF92EF92FF920F931F93CF93DF9379
:105B20008B01EA016115710521F0DB018C9311965F
:105B30009C93209739F09E01225031092332310580
:105B400008F0D8C07C016701BFEFCB1ADB0A560111
:105B5000F7016080862D90E00E94B12E892B11F014
:105B60007601F1CFFDE26F120AC0570182E0A80E64
:105B7000B11CD70111966C90772473940BC0BBE2D3
:105B80006B1207C05701E2E0AE0EB11CD7011196AF
:105B90006C90712CCE018F7E892B89F4B0E36B124F
:105BA00037C0F50180818F7D8835D1F46180F2E0C6
:105BB000AF0EB11C872D8260782EC0E1D0E0CA30D4
:105BC000D10551F1C031D10521F0C830D10599F48A
:105BD00009C0CC24CA94DC2CEC2CAFE0FA2E22C0F5
:105BE000209769F7C8E0D0E0CC24CA94DC2CEC2CD8
:105BF000FFE1FF2E17C06FEF7FEFCB019E0144271F
:105C000037FD4095542F0E94902C69017A010AC0FB
:105C10002097A9F6CAE0D0E0E9E9CE2EDC2CEC2CE6
:105C2000E9E1FE2EF50160E020E030E0A9014E013F
:105C3000AA2497FCA094BA2C1F0170ED572E560C85
:105C4000A9E0A51570F48FEB860D8A3118F499EC54
:105C5000592E06C08FE9860D8A3148F589EA582EFB
:105C6000560C852D90E08C179D070CF56F3FD9F0F1
:105C7000C216D306E406F50698F0C501B4010E94E9
:105C80006C2C9B01AC01852D90E0A0E0B0E0280FCA
:105C9000391F4A1F5B1F281739074A075B0710F493
:105CA0006FEF01C061E03196D1016C90C5CF011555
:105CB000110551F0662311F0319703C071FE04C045
:105CC0003297D801ED93FC9370FE07C05095409534
:105CD000309521953F4F4F4F5F4F67FF10C082E2D5
:105CE00090E090935E0680935D066FEF7FEF8FEFFD
:105CF0009FEF07C060E070E080E090E002C0B90173
:105D0000CA01DF91CF911F910F91FF90EF90DF902B
:105D1000CF90BF90AF909F908F907F906F905F904B
:105D20003F902F900895FC0188279927E8942191AE
:105D30002032E9F3293010F02E30C8F32B3241F035
:105D40002D3239F4689404C00E94E52E820F911D13
:105D5000219120532A30C0F31EF4909581959F4FD6
:105D60000895911150C0803219F089508550D0F7B4
:105D700008954AE953E00E94BE2E0895FA01A191C8
:105D8000B081009719F41097E1F0CD01DC01CD014D
:105D90000D90002011F4C00113C0FB0121912223BA
:105DA00019F02015D9F7F3CFFB012191201519F433
:105DB0001E92119606C02223C1F70D900020A1F774
:105DC000D001FA01A193B08308957AE0979F902DB6
:105DD000879F802D910D11240895F999FECF92BDD2
:105DE00081BDF89A992780B50895262FF999FECF9D
:105DF0001FBA92BD81BD20BD0FB6F894FA9AF99AE8
:105E00000FBE01960895992788270895F894FFCF2B
:105E100000005F06200001000000FF0002000200F9
:105E20000200020002000200020002000200020062
:105E300002000200020002000200028025000005AC
:105E4000400AA1204EA50020244EA52C2330C012CC
:105E500000001A400AA1204EA5001B1E27522C2329
:105E6000308025000005400AA1204EA50020244EC8
:105E7000A52C2330004B000006400AD0009D4900AD
:105E80007B289D492C233000E1000005400A450194
:105E9000D7DC03B81E0EBF00232E48E801008A405D
:105EA0000A6001555502AD1E20000023C801545858
:105EB0002074696D656F75742100596573004E6FAC
:105EC000002C00386368004E2F41002C205B005DE1
:105ED0002028002900486F70206368616E6E656C31
:105EE0002000204020007363616E6E6572206D6F2C
:105EF0006465004E4F5420454E41424C454400538A
:105F0000656E64696E672073657474696E6773206B
:105F1000746F2052580A00526573657474696E6715
:105F20002073657474696E6773206F6E2052580A0F
:105F30000041626F727465642065646974730A005D
:105F4000696E76616C69642073656C656374696FF2
:105F50006E000D0A496E76616C696420696E707519
:105F600074202D2064697363617264656421070085
:105F700053657474696E6773207361766564207409
:105F80006F20454550524F4D0A0052657665727438
:105F900065642073657474696E67732066726F6DD3
:105FA00020454550524F4D0A004C6F616465642096
:105FB000666163746F72792064656661756C747371
:105FC0000A004B657920616E64206368616E6E65BE
:105FD0006C732072616E646F6D697A65640A004F3C
:105FE00070656E4C52536E67205458207374617202
:105FF00074696E672000206F6E20485720006D6F17
:1060000064756C65206C6F636B65643F00342B3482
:10601000003800382B340031320031322B3400315B
:10602000360050504D0052535349005344410053E1
:10603000434C00525844005458440041494E004CCF
:10604000424545500053504B54524D005342555316
:106050000053554D44004C4C494E440000070B0C76
:1060600010111500B701FD020103030307030A0322
:106070000F03B701160A13223129120316031B035B
:106080001F03230327032B032F0335033C03410383
:1060900046035F025F025F025F0200000000922A77
:0A60A0009728382A652A4A2A872A21
:00000001FF
